:103E890000010C01010402011E030A960401320516
:103E9900030306006407010108000009015A0E0125
:103EA900010F000112006413010114013C1501FA0C
:103EB9001664FA17FFFF1D000720000724000227D8
:103EC90001012F013C30010132010335FFFF3603A7
:103ED900073CFFFF3DFFFF180002191E461A0002AA
:103EE9001B00022D32C82E0001FAFAFA1800001937
:103EF900FFFF1A00001B00002D32C82E0001FAFA3C
:103F0900FA18000019FFFF1A00001B00002DFFFF1F
:063F19002EFFFFFAFAFA88
:10004800900786E0FEA3E0FF7457BE0010D39F40E0
:100058000C903E8912001EE493F599804C90001490
:10006800E0D394044014900786E0FEA3E0FF903E9E
:100078008912001EE493F599802F900014E0D39420
:10008800034014900786E0FEA3E0FF903E9E120016
:100098001EE493F5998012900786E0FEA3E0FF9096
:1000A8003EB312001EE493F59990078612000E9055
:1000B8000786E0FEA3E0FF746C6F4E7003751300B3
:1000C80022900072E0B402087401900072F0D20C21
:1000D80090013AE090002AF090013BE090002BF06C
:1000E80090013CE090002CF0A20AB3401690013A2F
:1000F800E0700C90013BE0700690013CE0600280EB
:1001080002C20A90013AE0B4300F90013BE0B447D4
:100118000890013CE0643B60028004D20B8002C27C
:100128000BE558B40102800302024B900057E0F53A
:1001380066900062E0F568900063E0F569900074ED
:10014800E0F56A90007AE0900029F090007CE0F5F4
:100158006590007DE0F567900080E0F5649000818F
:10016800E0F563900090E0900041F0900091E090FD
:100178000042F0900092E0900043F0900093E090ED
:100188000044F0900094E0900045F0900095E090D5
:100198000046F0900096E0900047F0900097E090BD
:1001A8000048F0900099E0900033F090009AE090B9
:1001B8000034F090009BE0900035F090009CE090B7
:1001C8000036F0900079E0B4011790000A740FF03F
:1001D800A374FFF090000CE4F0A3F074029000798F
:1001E800F0900079E0B4035990000CE0FEA3E0FF22
:1001F80090000AE0FCA3E0FD1200037410123F9E79
:100208007408123F90EF900026F0EF700674FF908C
:100218000026F07400900079F090000BE090002721
:10022800F090000AE0900028F0900026E0900789FE
:10023800F0900027E090078AF0900028E090078B64
:10024800F0803F900081E07006755801756300A248
:100258000AB3402E90013AE090002AF090013BE06A
:1002680090002BF090013CE090002CF090002AE0E8
:10027800700C90002BE0700690002CE06002800269
:10028800C20AE5667003756602E568700375680260
:100298007E887F75E5668E048F05FF123F808C3956
:1002A8008D3AE56975F0FAA4FFAEF0E5688E048F23
:1002B80005FF123F808C3D8D3E90004FE0F5609029
:1002C800004DE0FE900069E0B5061890004CE0FE95
:1002D800900068E0B5060C90004BE0FE900059E0F5
:1002E8006E606F900069E07006900068E0600674C8
:1002F80000900059F0900069E0B402089000497439
:1003080001F08005900049E4F0900068E0B402082C
:1003180090004A7401F0800590004AE4F09000686B
:10032800E0600690004AE060028005756003800383
:10033800756004E559B55802D20C900068E0900049
:100348004CF0900069E090004DF0900059E090006A
:100358004BF0740190009EF0740190009FF07400BF
:100368009000A0F074009000A1F074009000A2F03A
:1003780074009000A3F074009000A4F07401900041
:10038800A5F074019000A6F074019000A7F0740025
:100398009000A8F074009000A9F074009000AAF0F2
:1003A80074009000ABF074019000ACF07401900000
:1003B800ADF074009000AEF074009000AFF07400DF
:1003C8009000B0F074009000B1F074009000B2F0AA
:1003D8007401900362F07401900363F07400900359
:1003E80064F07400900365F07400900366F0740084
:1003F800900367F07400900368F074009003A2F013
:1004080074019003A3F074009003A4F074009003A7
:10041800A5F074009003A6F074009003A7F0740090
:100428009003A8F074009003E2F074009003E3F0E6
:1004380074009003E4F074009003E5F074009003F6
:10044800E6F074009003E7F074009003E8F074019C
:10045800900422F07400900423F07400900424F0B7
:100468007400900425F07400900426F07400900441
:1004780027F07400900428F022E5B554F7F5B5E5A7
:10048800B554FDF5B5C292C287C290C207E5B5540E
:10049800FBF5B5755104E55104F55290004FE0F5B0
:1004A80060900025E4F0C209E5B554FEF5B5C28EAA
:1004B800758D00758B00754C00752600752500D26A
:1004C8008E22750A00750900AE09AF0A7457BE007E
:1004D800039F5003020587903E8912001EE4939003
:1004E800004E123FB60FBF00010EE0FC903E89128D
:1004F800001EECFEE493FFEEC39F5026AE09AF0A40
:100508000FBF00010E903E8912001EAE09AF0AE42B
:1005180093FC903E8912001EE49390004E123FB661
:10052800ECF0AE09AF0A903E8912001EE4939000E9
:100538004E123FB6E0FC903E8B12001EECFCE4939A
:10054800FDECD39D4019903E8B12001EE493FC9065
:100558003E8912001EE49390004E123FB6ECF0AEB6
:1005680009AF0A74022FFF50010E8E098F0A780A0C
:10057800740126F6500418E436F640030204D0222B
:10058800750A00750900AE09AF0A7415BE00039F0D
:100598005003020655903EE012001EE49390004E70
:1005A800123FB60FBF00010EE0FC903EE012001EA5
:1005B800ECFEE493FFEEC39F5026AE09AF0A0FBFCF
:1005C80000010E903EE012001EAE09AF0AE493FC53
:1005D800903EE012001EE49390004E123FB6ECF0FD
:1005E800AE09AF0A903EE012001EE49390004E124E
:1005F8003FB6E0FC903EE212001EECFCE493FDECFA
:10060800D39D4019903EE212001EE493FC903EE018
:1006180012001EE49390004E123FB6ECF0AE09AF04
:100628000A740F6F4E7006750A15750900AE09AF8A
:100638000A74022FFF50010E8E098F0A780A74017E
:1006480026F6500418E436F6400302058E22750A91
:1006580000750900AE09AF0A7415BE00039F500368
:10066800020723903EF512001EE49390004E123FBD
:10067800B60FBF00010EE0FC903EF512001EECFE26
:10068800E493FFEEC39F5026AE09AF0A0FBF0001E7
:100698000E903EF512001EAE09AF0AE493FC903EA0
:1006A800F512001EE49390004E123FB6ECF0AE092E
:1006B800AF0A903EF512001EE49390004E123FB62A
:1006C800E0FC903EF712001EECFCE493FDECD39D99
:1006D8004019903EF712001EE493FC903EF512007C
:1006E8001EE49390004E123FB6ECF0AE09AF0A74C8
:1006F8000F6F4E7006750A15750900AE09AF0A74BA
:10070800022FFF50010E8E098F0A780A740126F60F
:10071800500418E436F6400302065C22750A007598
:100728000900AE09AF0A7415BE00039F5003020703
:10073800F1903F0A12001EE49390004E123FB60F4C
:10074800BF00010EE0FC903F0A12001EECFEE4938D
:10075800FFEEC39F5026AE09AF0A0FBF00010E90EF
:100768003F0A12001EAE09AF0AE493FC903F0A123A
:10077800001EE49390004E123FB6ECF0AE09AF0AAB
:10078800903F0A12001EE49390004E123FB6E0FC20
:10079800903F0C12001EECFCE493FDECD39D401935
:1007A800903F0C12001EE493FC903F0A12001EE4D6
:1007B8009390004E123FB6ECF0AE09AF0A740F6F7B
:1007C8004E7006750A15750900AE09AF0A74022F36
:1007D800FF50010E8E098F0A780A740126F650041C
:1007E80018E436F6400302072A22054D22054C225A
:1007F800054EC2CF2290F800E4936406600280FEA2
:1008080075840175A70075FF80900788E4F075C9A5
:100818001075A70F75A1C775A70075D90075CEFF0C
:1008280075A70F75F1FE75F2FF75F33775F47875D6
:10083800A4BA75A5FF75A60775AE0075AFFF75D488
:100848008175D5FF75D6FF75D7FFC293C294C29143
:10085800E5B554BFF5B5E5B554DFF5B5E5B554EFE5
:10086800F5B5E5B5547FF5B5E5B554F7F5B5E5B596
:1008780054FDF5B575A70075A20175A14775F8096E
:1008880075BC0175BE0475BD6C75BE0775BDA075D8
:10089800BE0875BD0175BC0075BB1875BC2075BA5E
:1008A8000875E88075D11375A70F75E10575E20025
:1008B80075C740759700759780740A123F707597D1
:1008C800C0E5975420700280F8758F0275A700D292
:1008D800AF75980075A90C75A70F75AB4375ADFB7F
:1008E80075AC1E75A700758911758E00758C00751D
:1008F8008A00D2A9D28C758D00758B00D2ABD28EAE
:1009080075CD0075CC0075CA0075CB00D2ADC2CFCD
:10091800D2CA7591047592007593CD75EF0675D995
:100928004075CF01900786E4F0A3F07513007514A5
:1009380000C299D20AC20D12048174C8F51875173D
:10094800001226D775A70FE5FB90001AF0E5FA907C
:10095800001BF0E5F990001CF075A70090F800E482
:1009680093F50812280E122D48900789E09000266A
:10097800F090078AE0900027F090078BE09000281D
:10098800F090078CE0900029F090078DE0F56690D4
:10099800078EE0F56890078FE0F569900790E0F51D
:1009A8006A900791E0F565900792E0F567900793E4
:1009B800E0F564900794E0F563900795E090002ACD
:1009C800F0900796E090002BF0900797E090002CAD
:1009D800F0900798E0900041F0900799E09000426D
:1009E800F090079AE0900043F090079BE090004455
:1009F800F090079CE0900045F090079DE09000463D
:100A0800F090079EE0900047F090079FE090004824
:100A1800F09007A0E0900033F09007A1E090003438
:100A2800F09007A2E0900035F09007A3E090003620
:100A3800F07400900082F090013AE0700C90013B55
:100A4800E0700690013CE060028004C20A8002D295
:100A58000A90F807E493900021F0900021E0440AFE
:100A6800900021F0900021E054FE900021F07406DF
:100A7800900012F07402900013F090F802E4939042
:100A88000014F07403900015F07403900016F074CD
:100A98001A900017F07405900018F0900014E0B454
:100AA80004067404900018F0900014E0B40306746F
:100AB80003900018F07405900019F090F804E4937E
:100AC80090001DF0740090001EF090F805E49390DB
:100AD800001FF090F806E493900020F074FF900057
:100AE80022F0745A900125F07446900126F0742083
:100AF800900127F07434900128F07448900129F08F
:100B0800745090012AF0743290012BF074349001E3
:100B18002CF0742090012DF0743590012EF0742D76
:100B280090012FF07453900130F0746F900131F000
:100B3800746C900132F07420900133F090007AE0E8
:100B4800D394014006740090007AF07558017559E5
:100B580001740390004CF01200C91204CA900014EA
:100B6800E0B404051206568011900014E0D39404F2
:100B780040051205888003120724122703E5B5549F
:100B8800FEF5B5900025E4F0900786E4F0A3F07533
:100B98002400752300754800752A007529007549D9
:100BA80000753200753100754A007554007555009E
:100BB800755A0075510475520175343C75330075CA
:100BC8007000756F007571CD7556007557007543C7
:100BD80000754400754500754600755B0075470053
:100BE800754200754100900006E4F0A3F0900008FB
:100BF800E4F0A3F0755E00755F0090000E74FDF0E0
:100C0800A374E8F0900023E4F07464900024F0C228
:100C180000D201C202D203754D00756D00C297C2A1
:100C2800A0C296C295C2A2C20C7E017F0090002885
:100C3800E0123F9E900027E02FFF50010E90000A1F
:100C4800EEF0A3EFF0900026E0700674FF90002607
:100C5800F090000AE0FEA3E0FFEFD394FFEE940FBC
:100C6800400790000AE4F0A3F07400900071F0745B
:100C780000900079F07400900082F0740090008D6C
:100C8800F074009000B4F0E5677003756704743A77
:100C980090074EF074FD90074FF09003D4E0900455
:100CA80014F0D2B0D2B7D2A7D2A6D2B1D2A3C2077B
:100CB800A2B6B39204A2B3B39205D29CD2EC75CF7C
:100CC80001A298B34005C2981230ACE5136006A2A1
:100CD80099B3B340028005C29912361CE514640129
:100CE8006005E514B4040280D5E54DD39405400CA5
:100CF800E55AC394C85002055A754D00E571C3946E
:100D0800F0501A786F12003FAE6FAF70EFD394E8CF
:100D1800EE940340080571757000756F00C28E7EF1
:100D2800047F00E54C123F9EE58D75F004A4FDACF0
:100D3800F0EF2DFDEE3CFCE58B75F04084FF7E0066
:100D4800ED2FFFEC3EFE8E258F26D28EA2B6300404
:100D580001B35003020E99A2B6300401B350030246
:100D68000E99A2B640670554A20D400575FFA0D2A2
:100D78000DE5B54401F5B5900024E4F0E554D395AC
:100D88006640487C887D75AE25AF26123DA88E2327
:100D98008F24E5482FFF50010E7401123F908E23D7
:100DA8008F24852448755401C28E758D00758B007B
:100DB800754C00D28E7403BE00039F500690002528
:100DC8007401F0E543B40603754300D204A2B6B338
:100DD8005003020E99C20490006BE0601812375D50
:100DE800A200B34008E5B54408F5B58006E5B5545A
:100DF800F7F5B58002C20090006EE060181238B2B4
:100E0800A202B34008E5B54402F5B58006E5B5543D
:100E1800FDF5B58006E5B554FDF5B5A207B3400468
:100E2800D2968002C296900059E06004D295800262
:100E3800C29590004AE0B40104D2978002C297900C
:100E48000049E0B40104D2A08002C2A0A209B340C4
:100E580004D2A28002C2A2900018E0FE900014E022
:100E6800C39E4009900014E0D39408400974FB9095
:100E78000023F012048190001DE0601590001DE031
:100E8800FE900017E06E600974FE900023F01204D3
:100E980081C2CA7E017F00E54E123F9EE5CD2FFF3D
:100EA80050010E8E278F28D2CAE565B401489000FC
:100EB8000EE0FCA3E0FDEFC39DEE9C4039B208E5CF
:100EC8002A45296013A208B34008E5B54404F5B5DE
:100ED8008006E5B554FBF5B590000EE0FEA3E0FFF3
:100EE800900010E0FCA3E0FDEF2DFDEE3CFC90002F
:100EF8000EECF0A3EDF0A2B3300501B35003020FDE
:100F0800E7A2B3300501B35003020FE7A2B35003C1
:100F1800020FE00555A20D400575FFA0D20DE5B5FD
:100F28004401F5B5900024E4F0E555D395685003E5
:100F3800020FDE7CEA7D60AE27AF28123DA88E291D
:100F48008F2AE569123F9E74FF8E048F05FF123FBA
:100F5800808C298D2AE5492DFD50010C74018C06E1
:100F68008D07123F908E298F2A852A49A209B340FE
:100F7800157464123F9E900067E08E048F05FF127F
:100F88003F808C298D2A75550190000EE0FEA3E064
:100F9800FFAC27AD2812000390000EEEF0A3EFF08F
:100FA800E567FF123F80740AFF123F8090007BE0E4
:100FB8008C068D07123F9E74148E048F05FF123F16
:100FC80080900010ECF0A3EDF0C2CA75CD0075CC8E
:100FD80000754E00D2CAD205A2B3B34002C2059032
:100FE8000025E0B40107E556C3940640030215F353
:100FF800E56D9026B6F8282873900059E0C394024E
:101008004003021155E551D394015003021155E5EF
:101018005175F040A4FFAEF090031212001EE0C319
:1010280095455018E55175F040A4FFAEF0900311B6
:1010380012001EE0F52E752D00021155E55175F0D0
:1010480040A4FFAEF090031012001EE0C395454087
:10105800030210F1E55175F040A4FFAEF0900311C2
:1010680012001EE55175F040A4FFAEF0E0FC9003BD
:101078000F12001EECFEE0FFEEC39FFEE5518E044A
:1010880075F040A4FFAEF090031012001EE0F404C7
:1010980025458C0088F0A4FFAEF0E5518F048E053D
:1010A80075F040A4FFAEF090031212001EE55175D2
:1010B800F040A4FFAEF0E0FA90031012001EEAFE22
:1010C800E0FFEEC39FFECDCCCD8E07123F80E551E9
:1010D80075F040A4FFAEF090030F12001EE02DFD46
:1010E80050010C8C2D8D2E8064E55175F040A4FFC5
:1010F800AEF090030F12001EE55175F040A4FFAE4C
:10110800F0E0FC90030E12001EECFEE0FFEEC39F21
:101118008545F0A4FFAEF0E5518F048E0575F040CB
:10112800A4FFAEF090031012001EE0FECDCCCD8ED1
:1011380007123F80E55175F040A4FFAEF090030E12
:1011480012001EE02DFD50010C8C2D8D2E756D01A9
:101158000215F3900059E0C394024003021308906B
:10116800004FE0D3955150030212B1E55175F0409C
:10117800A4FFAEF090031812001EE0C39545501866
:10118800E55175F040A4FFAEF090031712001EE081
:10119800F52C752B000212B1E55175F040A4FFAE95
:1011A800F090031612001EE0C39545400302124D4D
:1011B800E55175F040A4FFAEF090031712001EE54C
:1011C8005175F040A4FFAEF0E0FC90031512001E2C
:1011D800ECFEE0FFEEC39FFEE5518E0475F040A4DF
:1011E800FFAEF090031612001EE0F40425458C00B3
:1011F80088F0A4FFAEF0E5518F048E0575F040A489
:10120800FFAEF090031812001EE55175F040A4FFE0
:10121800AEF0E0FA90031612001EEAFEE0FFEEC3FD
:101228009FFECDCCCD8E07123F80E55175F040A4CE
:10123800FFAEF090031512001EE02DFD50010C8C3E
:101248002B8D2C8064E55175F040A4FFAEF090031F
:101258001512001EE55175F040A4FFAEF0E0FC90B9
:10126800031412001EECFEE0FFEEC39F8545F0A4B8
:10127800FFAEF0E5518F048E0575F040A4FFAEF087
:1012880090031612001EE0FECDCCCD8E07123F80D3
:10129800E55175F040A4FFAEF090031412001EE073
:1012A8002DFD50010C8C2B8D2CE551B40122E560ED
:1012B800D39401401BE551C395565014E545C3949A
:1012C80005500D90035FE0A829B80006952A400252
:1012D8008003755102E551B5602290004FE0D39527
:1012E800514019E55175F040A4FFAEF09003171274
:1012F800001EE0A823B8000695244002800205607D
:10130800756D020215F3900059E0B4022AE5517593
:10131800F040A4FFAEF090031712001EE0F52C7504
:101328002B00E55175F040A4FFAEF090030E1200BB
:101338001EE0F52E752D00900059E0B4030F9000C3
:1013480051E0F52C752B00752E00752D00756D0379
:101358000215F3E55175F040A4FFAEF0900320129A
:10136800001EE0C3955A400302142A900049E07019
:1013780036E551D394014029AE23AF24AC2DAD2ED0
:10138800EDD39FEC9E401AE55175F040A4FFAEF0F6
:1013980090031E12001EE0A829B80005D3952A5014
:1013A80002800215518034E551D394024029AE23BE
:1013B800AF24AC2DAD2EEDD39FEC9E401AE55175B0
:1013C800F040A4FFAEF090031E12001EE0A829B85A
:1013D8000005D3952A500280021551E551C3956046
:1013E800502FE551C395565028AE23AF24AC2BADF2
:1013F8002CEFD39DEE9C4019E55175F040A4FFAE4B
:10140800F090031F12001EE0A829B80006952A4094
:101418000280020551C290E55165526005C2077508
:101428005A00756D040215F3E55175F040A4FFAE3E
:10143800F090031A12001EE0B40117E55175F04050
:10144800A4FFAEF090032012001EE0240AC3955AB0
:101458004003021500753064752F00A207B3500BC6
:10146800900060E02405C395454003021500E5514E
:1014780075F040A4FFAEF090031D12001EE0C39566
:10148800454064E55175F040A4FFAEF090031C128E
:10149800001EE55175F040A4FFAEF0E0FC90031B80
:1014A80012001EECFEE0FFEEC39F8545F0A4FFAEE0
:1014B800F0E5518F048E0575F040A4FFAEF090035F
:1014C8001D12001EE0FECDCCCD8E07123F80E551E7
:1014D80075F040A4FFAEF090031B12001EE02DFD36
:1014E80050010C8C2F8D30AE23AF24AC2FAD30EFD4
:1014F800D39DEE9C4002D207756D050215F3E551A8
:10150800B40109900059E0C3940240030215D39036
:101518000358E0D3954550030215D3900356E0C312
:1015280095455040900357E0FE900355E0F4042E93
:10153800FE900356E0F40425458E0088F0A4FFAE23
:10154800F0900358E0FC900356E0F4042C8E048FCE
:1015580005FF123F80900355E02DFD50010C8C2BA8
:101568008D2C802C900355E0FE900354E0F4042E5B
:101578008545F0A4FFAEF0900356E08E048F05FF7A
:10158800123F80900354E02DFD50010C8C2B8D2CC4
:10159800E551C39560502FE551C395565028AE23A9
:1015A800AF24AC2BAD2CEFD39DEE9C4019E55175C3
:1015B800F040A4FFAEF090031F12001EE0A829B867
:1015C8000006952A40028003755102900049E0B454
:1015D8000106E551640160028003755102E5516519
:0B15E800526005C207755A00756D00C7
:1026B60002100102115B02130E02135B02143002B8
:0226C6001506F7
:1015F300900050E02402A823B80007D395244002AA
:10160300C207900025E0B40109900059E0C3940398
:101613004003021779900049E060030216C9E551BF
:10162300D394014034E55175F040A4FFAEF090032C
:101633001412001EE0A823B8001FD39524401AE516
:101643005175F040A4FFAEF090031F12001EE0A8F6
:1016530029B80005D3952A500280021551E551D3CC
:101663009401402FE55175F040A4FFAEF0900312B2
:1016730012001EE0C39545501AE55175F040A4FFD2
:10168300AEF090031E12001EE0A829B80005D39502
:101693002A500280021551E551D394014021E551AE
:1016A300D39556401AE55175F040A4FFAEF0900370
:1016B3001E12001EE0A829B80005D3952A50028007
:1016C30002155102176EE551D394024034E551756A
:1016D300F040A4FFAEF090031412001EE0A823B85C
:1016E300001FD39524401AE55175F040A4FFAEF0D6
:1016F30090031F12001EE0A829B80005D3952A50B5
:101703000280021551E551D39402402FE55175F043
:1017130040A4FFAEF090031212001EE0C3954550A3
:101723001AE55175F040A4FFAEF090031E12001E9F
:10173300E0A829B80005D3952A500280021551E587
:1017430051D394024021E551D39556401AE5517582
:10175300F040A4FFAEF090031E12001EE0A829B8CB
:101763000005D3952A500280021551E55165526058
:1017730005C207755A00900060E0D3954550099063
:101783000054E0C395455002C207900059E070032E
:101793000219DCA2A5B34008A2A4B340030219C5F1
:1017A300AE35AF367441D39F749C9E400578351295
:1017B300003FAE35AF36EFB48806EEB413028003B4
:1017C3000219A2A2A55003021865900059E0B401C2
:1017D3000B90004FE0D3956040020560900059E004
:1017E300B40253E55175F040A4FFAEF0900320120C
:1017F300001EE0C3955A503E90004FE0D3955140F0
:1018030020E551C395565019E55175F040A4FFAE3C
:10181300F090031412001EE0A823B800069524409C
:10182300028002055190004FE0F560E5516552607A
:1018330005C207755A00900059E0B4032590004F84
:10184300E0D395514007E551C39556400280020508
:101853005190004FE0F560E55165526005C2077590
:101863005A00A2A450030219A2900059E0B4016ED9
:10187300900049E07035E551D394014029E5517555
:10188300F040A4FFAEF090031E12001EE0A829B89A
:10189300000FD3952A400A1551755A00855160806F
:1018A3000385516080037560018033E551D3940251
:1018B3004029E55175F040A4FFAEF090031E1200DD
:1018C3001EE0A829B8000FD3952A400A1551755A6E
:1018D300008551608003855160800375600290002C
:1018E30059E0D394015003021996E55175F040A4D1
:1018F300FFAEF090032012001EE0C3955A4003028E
:101903001996900049E07041E551D394014034E5C4
:101913005175F040A4FFAEF090031112001EE0A831
:1019230023B8001FD39524401AE55175F040A4FF56
:10193300AEF090031E12001EE0A829B80005D3954F
:101943002A500280021551803FE551D3940240345E
:10195300E55175F040A4FFAEF090031112001EE0B4
:10196300A823B8001FD39524401AE55175F040A46D
:10197300FFAEF090031E12001EE0A829B80005D3A5
:10198300952A500280021551E55165526005C20740
:10199300755A00E556B40704055E8003755E00E5DD
:1019A30063B4010EAE35AF36EF64407005EE649C50
:1019B3006002800EA2A54003755801A2A4400375DE
:1019C3005802A2A5B3B35006A2A4B3B34002800643
:1019D300753600753500021ACAA2A5B34008A2A441
:1019E300B34003021AB6AE35AF367441D39F749C2D
:1019F3009E4005783512003FAE35AF36EFB488060A
:101A0300EEB413028003021AB6A2A5406F900068D9
:101A1300E0605A90004AE0B4010790004AE4F08085
:101A23000690004A7401F090004AE0700575600367
:101A3300800375600490004AE0B40104D2978002E9
:101A4300C297E551B4041AE55175F040A4FFAEF016
:101A530090031E12001EE0A829B80005D3952A5052
:101A6300028008755103C207755A0080037560042C
:101A7300E556B40704055E8003755E00A2A44033F7
:101A8300900069E06021900049E0B40107900049AB
:101A9300E4F080069000497401F0900049E0B4013D
:101AA30004D2A08002C2A0E556B40704055E8003F9
:101AB300755E00A2A5B3B35006A2A4B3B3400280DF
:101AC30006753600753500E5586559600690008245
:101AD300E06003021C52C29C751400751300C2CA55
:101AE300E5589026C8F82828738012122D48800DD7
:0D1AF300122E218008122EFA8003122FD32C
:0F26C800021AEC021AEE021AF3021AF8021AFDB5
:101B0000900029E090007AF0E566900057F0E568D3
:101B1000900062F0E569900063F0E56A900074F06F
:101B2000E56590007CF0E56790007DF0E56490004D
:101B300080F0E563900081F090002AE090013AF097
:101B400090002BE090013BF090002CE090013CF0E5
:101B5000900041E0900090F0900042E0900091F001
:101B6000900043E0900092F0900044E0900093F0E9
:101B7000900045E0900094F0900046E0900095F0D1
:101B8000900047E0900096F0900048E0900097F0B9
:101B9000900033E0900099F0900034E090009AF0CB
:101BA000900035E090009BF0900036E090009CF0B3
:101BB0007400900082F0745A900125F074469001F0
:101BC00026F07420900127F07434900128F07448B6
:101BD000900129F0745090012AF0743290012BF09A
:101BE000743490012CF0742090012DF07435900124
:101BF0002EF0742D90012FF07453900130F0746F1B
:101C0000900131F0746C900132F07420900133F047
:101C10009003D4E0900414F0743A90074EF074FDF1
:101C200090074FF01200C9900004E4F0A3F0900078
:101C3000067475F0A37430F09000087475F0A37406
:101C400030F0855859D2CA754C00D29C741B900054
:101C500023F0E556C394065005E551B5520280675E
:101C6000C207E55175F040A4FFAEF09003221200C8
:101C70001EE030E003D38001C39293E55175F0403C
:101C8000A4FFAEF090032312001EE030E003D380E7
:101C900001C39294E55175F040A4FFAEF090032487
:101CA00012001EE030E003D38001C39291855152AF
:101CB000AE29AF2A7405BE00039F5007E545D394B3
:101CC0000550028002D290E556D394055003021DC0
:101CD000D1C207E551D394014073E55175F040A49A
:101CE000FFAEF090031E12001EE0A829B80007D333
:101CF000952A40021551E5516552604EE55175F047
:101D000040A4FFAEF090032212001EE030E003D3A7
:101D10008001C39293E55175F040A4FFAEF09003AB
:101D20002312001EE030E003D38001C39294E551FA
:101D300075F040A4FFAEF090032412001EE030E0E6
:101D400003D38001C39291855152021DD1E556B44F
:101D500006279000ACE030E003D38001C39293905B
:101D600000ADE030E003D38001C392949000AEE078
:101D700030E003D38001C39291E556B40727900069
:101D8000A5E030E003D38001C392939000A6E03039
:101D9000E003D38001C392949000A7E030E003D326
:101DA0008001C39291E556B4082790009EE030E090
:101DB00003D38001C3929390009FE030E003D3806F
:101DC00001C392949000A0E030E003D38001C3925D
:101DD00091900072E06058E54575F00284FF7E0046
:101DE00090014E12001EE0F55CE54775F00A84FF95
:101DF0007E0090024E12001EE0F55DE55C255DD38D
:101E00009464400BE55C255DC39464F55C800375C8
:101E10005C00E55C75F00284FF7E008F5CEFC3948C
:101E2000335007EF24CDF55C8003755CFF801CE523
:101E30004575F00284FF7E0090014E12001EE07591
:101E4000F00284FF7E00EF24CDF55CE595C3955C40
:101E50004004C2928002D292A207B34005E556B474
:101E600007037571CDE595C395714004C287800263
:101E7000D287E543C394064003022475A2EDB35014
:101E800003022475C2EDE5436003021FD77E017F84
:101E900000E5BE123F9EE5BD2FFF50010E900000F1
:101EA000EEF0A3EFF0900029E0B401177E0F7FFF62
:101EB000900000E0FCA3E0FD120003900000EEF0B3
:101EC000A3EFF0900079E0B4025B900000E0FEA385
:101ED000E0FF90000AE0FCA3E0FDEDD39FEC9E4004
:101EE0000F900000E0F8A3E090000AC8F0A3C8F04B
:101EF000900000E0FEA3E0FF90000CE0FCA3E0FDFA
:101F0000EFD39DEE9C400F900000E0F8A3E090001E
:101F10000CC8F0A3C8F0900000E0FEA3E0FF74043A
:101F2000123F908F44900079E07060900000E0FED6
:101F3000A3E0FF90000AE0FCA3E0FDEFD39DEE9C40
:101F4000400D120003900000EEF0A3EFF080079028
:101F50000000E4F0A3F0900000E0FEA3E0FF7410A6
:101F6000123F9E900026E08E048F05FF123F809066
:101F70000000ECF0A3EDF07400D39D74019C4008C8
:101F8000900001E0F54480037544FFE54475F00AD4
:101F9000A4FFAEF074198E048F05FF123F808D45AB
:101FA000ED2532FFAE3150010E7401123F908F4586
:101FB000854532753100EFD39462400375456290D8
:101FC0000072E064016006900066E06002800575C2
:101FD0004301800375BB17E543B40102800302206F
:101FE000C77E017F00E5BE123F9EE5BD2FFF500179
:101FF0000E900000EEF0A3EFF0900072E0B4017ECE
:10200000E53445336025AC33AD341DBDFF011C8F75
:10201000028E038C068D07903AD412002EE493FEB4
:10202000740193FFEFC39AEE9B4002800578331250
:102030003FC8AE33AF3474B3BE0025D39F40219068
:102040000000E0FCA3E0FD0FBF00010E903AD412A7
:10205000002EE493FE740193FFEDC39FEC9E4002BB
:102060008005783312003FAE33AF34E56A123F9EED
:1020700074648E048F05FF123F808D47803390007B
:1020800066E0602D900000E0FEA3E0FFEFD3940037
:10209000EE9408400F900066E0B40104C20980028B
:1020A000D209800D900066E0B40104D2098002C21A
:1020B00009900072E064026006900066E0600575B9
:1020C000BB168003754302E543B40202800302217C
:1020D000B57E017F00E5BE123F9EE5BD2FFF50019A
:1020E0000E900000EEF0A3EFF0900072E0B4027EDC
:1020F000E53445336025AC33AD341DBDFF011C8F85
:10210000028E038C068D07903C3E12002EE493FE57
:10211000740193FFEFC39AEE9B400280057833125F
:102120003FC8AE33AF3474B3BE0025D39F40219077
:102130000000E0FCA3E0FD0FBF00010E903C3E124A
:10214000002EE493FE740193FFEDC39FEC9E4002CA
:102150008005783312003FAE33AF34E56A123F9EFC
:1021600074648E048F05FF123F808D47803390008A
:1021700066E0602D900000E0FEA3E0FFEFD3940046
:10218000EE9408400F900066E0B40104C20980029A
:10219000D209800D900066E0B40104D2098002C229
:1021A00009900072E07003754700900066E07002CD
:1021B000C20975BB1FE543B403457E017F00E5BE40
:1021C000123F9EE5BD2FFF50010E900000EEF0A3E0
:1021D000EFF07409123F9E74E68E048F05FF123FE4
:1021E000808C418D42E54A2DFD50010C74018C0616
:1021F0008D07123F908E418F4285424A75BB19E58B
:1022000043B40402800302235D7E017F00E5BE1219
:102210003F9EE5BD2FFF50010E900000EEF0A3EFB2
:10222000F07404123F908F4BE564B4010280030206
:1022300022EA756B00756B00E56BD39407400302CF
:1022400022D7E56B900041123FB6E0D3954B501A70
:10225000E56B900041123FB6E0F404254BFEE56BC0
:10226000900037123FB6EEF08017E56B90004112F8
:102270003FB6E0C3954BFEE56B900037123FB6EEDC
:10228000F0E56BC394044009900084E0C3956B5063
:102290003BE56B6029E56B900037123FB6FEE0FF2F
:1022A000EE90003FE0D39F4013E56B900037123F64
:1022B000B6E090003FF0E56B900040F0800E90009B
:1022C00037E090003FF07400900040F0786B7401AC
:1022D00026F64003022238900040E0F4042408F57A
:1022E00056E556D394054002C290E564D39401406C
:1022F0002FE54BD3946E4004D20E8002C20E755669
:1023000005E564B40205A20EB340028003755607CA
:10231000E564B40306A20EB3B3400280037556070A
:10232000E55765566008E55104F552855657E55660
:10233000B40708E5B54480F5B58006E5B5547FF5EA
:10234000B5E55664066005E556B40808E5B54410E1
:10235000F5B58006E5B554EFF5B575BB13E543B4A7
:10236000050280030224717E017F00E5BE123F9EBC
:10237000E5BD2FFF50010E900000EEF0A3EFF074CA
:1023800004123F908F46E563B40202800302246E7C
:10239000756B00756B00E56BD39403400302242535
:1023A000E56B900033123FB6E0D39546501AE56BCB
:1023B000900033123FB6E0F4042546FEE56B900032
:1023C0002D123FB6EEF08017E56B900033123FB64A
:1023D000E0C39546FEE56B90002D123FB6EEF0E5AA
:1023E0006B6029E56B90002D123FB6FEE0FFEE908A
:1023F0000031E0D39F4013E56B90002D123FB6E013
:10240000900031F0E56B900032F0800E90002DE0EE
:10241000900031F07400900032F0786B740126F671
:102420004003022396900082E07043E52A4529602C
:1024300036E558C39403500A900032E004C3940375
:1024400040028007900032E004F558E558D394022A
:10245000400A900032E004D39402500280079000BA
:1024600032E004F5588007900032E004F55875BB5F
:10247000180543D2ECE55ED394045003022576752B
:10248000CF01C292AE35AF367488D39F74139E408D
:1024900005A2A5B34014AE35AF367488D39F74132C
:1024A0009E4005A2A4B340028048783512003FAE9A
:1024B00035AF36EFB4883BEEB41337A2A5B350095D
:1024C00090004FE0D395515002800405518011A235
:1024D000A5B3500890004FE0655160028002D2071A
:1024E000A2A4B35007E551D39401500280041551C2
:1024F000C207A2A5B3B35006A2A4B3B3400280069C
:10250000753600753500E5516552604EE55175F040
:1025100040A4FFAEF090032212001EE030E003D38F
:102520008001C39293E55175F040A4FFAEF0900393
:102530002312001EE030E003D38001C39294E551E2
:1025400075F040A4FFAEF090032412001EE030E0CE
:1025500003D38001C39291855152A2074005757142
:10256000CD80037571FFE595C395714004C28780E6
:1025700002D28702247FA20DB3500DAE25AF267480
:10258000E8C39F74039E4002800575FFA0D20DAE84
:1025900025AF26EFD39420EE944E500302268A12E4
:1025A0000481C28E758D00758B00754C00D28EC271
:1025B00007757000756F007571CD75510475240035
:1025C000752300755400755A00C296900059E0605A
:1025D00004D2958002C29590004AE0B40104D297DB
:1025E0008002C297900049E0B40104D2A08002C2E8
:1025F000A0A209B34004D2A28002C2A290006BE064
:10260000601812375DA200B34008E5B54408F5B57F
:102610008006E5B554F7F5B58002C20090006EE083
:1026200060181238B2A202B34008E5B54402F5B50D
:102630008006E5B554FDF5B58006E5B554FDF5B564
:1026400090000E74FDF0A374E8F0E543B406037542
:102650004300900025E4F0752600752500758D0077
:10266000758B00754C00900024E0C39403500890D3
:102670000024E004F080067403900024F09000240D
:10268000E0B40306E5B554FEF5B5AE27AF28EFD3A9
:102690009410EE9427401CC2CA75CD0075CC00750D
:1026A0002800752700D2CA754E00752A00752900CA
:0626B000755500020CC686
:103A64000000010001320164019601960200021275
:103A740002240200020003000340038003C0040088
:103A84000440048004C00500060006000600060089
:103A9400060006000600060000FF013101630195DF
:103AA40001FF01FF0211022302FF02FF02FF033F95
:103AB400037F03BF03FF043F047F04BF04FF05FF2C
:103AC40006FF06FF06FF06FF06FF06FF06FF06FFCA
:103AD4000FAA0FA50F9F0F9A0F940F8D0F870F80BA
:103AE4000F780F710F680F600F570F4E0F450F3B84
:103AF4000F300F250F1A0F0E0F020EF50EE80EDB16
:103B04000ECC0EBE0EAE0E9F0E8E0E7D0E6C0E5A99
:103B14000E470E340E200E0C0DF70DE20DCB0DB535
:103B24000D9D0D850D6D0D540D3A0D200D050CE9FF
:103B34000CCE0CB10C940C760C580C3A0C1B0BFBF1
:103B44000BDB0BBB0B9A0B790B570B350B130AF1E1
:103B54000ACE0AAB0A870A640A400A1C09F809D487
:103B640009B0098C09670943091F08FB08D608B284
:103B7400088E086A0846082307FF07DC07B907967A
:103B840007730751072F070D06EC06CA06AA068914
:103B940006690649062A060A05EC05CD05B0059214
:103BA40005750558053C0520050504EA04CF04B550
:103BB400049C04820469045104390422040B03F4B0
:103BC40003DE03C803B2039D038903750361034D38
:103BD400033B03280316030402F202E102D102C0EC
:103BE40002B002A0029102820273026502570249E6
:103BF400023C022F02220216020901FD01F201E633
:103C040001DB01D001C601BB01B101A7019D0194F3
:103C1400018B018201790170016801600158015032
:103C24000148014101390132012B0125011E01180E
:103C34000111010B010500FF00FA0FA60FA00F9957
:103C44000F920F8B0F840F7C0F740F6B0F620F5842
:103C54000F4E0F430F380F2C0F1F0F120F050EF7C7
:103C64000EE80ED80EC80EB70EA50E930E800E6C7D
:103C74000E580E420E2C0E150DFD0DE40DCB0DB19C
:103C84000D950D790D5D0D3F0D200D010CE10CC05E
:103C94000C9E0C7C0C590C350C100BEA0BC40B9EBF
:103CA4000B760B4F0B260AFD0AD40AAA0A800A5582
:103CB4000A2A09FF09D409A8097C0950092508F929
:103CC40008CD08A10875084A081E07F307C8079D10
:103CD40007730749072006F706CE06A6067E065791
:103CE4000630060A05E405BF059B05770554053231
:103CF400051004EF04CE04AE048F0471045304359C
:103D0400041903FD03E203C703AD0394037B0363B8
:103D1400034B0334031E030802F302DE02CA02B695
:103D240002A30291027F026D025C024C023C022C4F
:103D3400021D020E020001F201E401D701CA01BE14
:103D440001B101A6019A018F0185017A0170016612
:103D5400015D0153014A0141013901310129012168
:103D640001190112010B010400FD00F700F000EA43
:103D740000E400DE00D900D300CE00C900C400BFB7
:103D840000BA00B500B100AD00A800A400A0009CDA
:103D9400009900950091008E008A008700840081BC
:043DA400007E007B22
:1026D700751A00751900AE19AF1AAC17AD18EDC30E
:1026E7009FEC9E401674FF123F7075CF01781A74E5
:1026F7000126F6500418E436F650DB22900786E4EC
:10270700F0A3F0751000750F00751300751400C263
:102717000FD21022C2AF75D900758F0375B7A57593
:10272700B7F190F800E4F0758F0175B7A575B7F1AB
:10273700E50890F800F075B7A575B7F190F801E4D2
:10274700F075B7A575B7F190079DE090F802F075A1
:10275700B7A575B7F19007A1E090F803F075B7A595
:1027670075B7F190079EE090F804F075B7A575B7B7
:10277700F190079FE090F805F075B7A575B7F19050
:1027870007A0E090F806F075B7A575B7F19007A216
:10279700E090F807F0758F0075D940D2AF22900707
:1027A70088E0B4AB61C2AF75D90075B62275F52262
:1027B700758F0375B7A575B7F1740090F600F075BE
:1027C7008F01750A00750900AE09AF0A7413BE00C0
:1027D700279F402475B7A575B7F190078912001E8A
:1027E700E0FC90F60012001EECF0780A740126F661
:1027F700500418E436F650D0758F0075F51175B68C
:102807002075D940D2AF22C2AF75D90075F52275B0
:102817000A00750900AE09AF0A7413BE00229F4073
:102827001F90F60012001EE493FC90078912001E09
:10283700ECF0780A740126F6500418E436F650D501
:1028470075F51175D940D2AF22900788E0B4AA0276
:10285700800302298DC2AF75D90075B62275F5229E
:10286700758F0375B7A575B7F1740090EE00F07515
:10287700B7A575B7F1740090F000F075B7A575B7F7
:10288700F1740090F200F075B7A575B7F174009078
:10289700F400F0758F01750A00750900AE09AF0ADB
:1028A70074FFC39F74019E402475B7A575B7F19057
:1028B700004E12001EE0FC90EE0012001EECF078B5
:1028C7000A740126F6500418E436F650CF750A004C
:1028D700750900AE09AF0A74FFC39F74019E4024B7
:1028E70075B7A575B7F190024E12001EE0FC90F087
:1028F7000012001EECF0780A740126F6500418E462
:1029070036F650CF750A00750900AE09AF0A74FF95
:10291700C39F74019E402475B7A575B7F190044E07
:1029270012001EE0FC90F20012001EECF0780A7410
:102937000126F6500418E436F650CF750A007509DB
:1029470000AE09AF0A74FFC39F74019E402475B798
:10295700A575B7F190064E12001EE0FC90F4001228
:10296700001EECF0780A740126F6500418E436F6D7
:1029770050CF758F0075F51175B62075D940D2AF58
:10298700743A90074EF022900788E0B4AA028003B9
:10299700022ACBC2AF75D90075B62275F522758F9D
:1029A7000375B7A575B7F1740090E600F075B7A584
:1029B70075B7F1740090E800F075B7A575B7F174B5
:1029C7000090EA00F075B7A575B7F1740090EC00B8
:1029D700F0758F01750A00750900AE09AF0A74FF1B
:1029E700C39F74019E402475B7A575B7F190004E3B
:1029F70012001EE0FC90E60012001EECF0780A744C
:102A07000126F6500418E436F650CF750A0075090A
:102A170000AE09AF0A74FFC39F74019E402475B7C7
:102A2700A575B7F190024E12001EE0FC90E8001267
:102A3700001EECF0780A740126F6500418E436F606
:102A470050CF750A00750900AE09AF0A74FFC39F1E
:102A570074019E402475B7A575B7F190044E120016
:102A67001EE0FC90EA0012001EECF0780A740126C2
:102A7700F6500418E436F650CF750A00750900AE13
:102A870009AF0A74FFC39F74019E402475B7A575EB
:102A9700B7F190064E12001EE0FC90EC0012001EEB
:102AA700ECF0780A740126F6500418E436F650CF95
:102AB700758F0075F51175B62075D940D2AF743A88
:102AC70090074EF022900788E0B4AA028003022CF8
:102AD70009C2AF75D90075B62275F522758F0375D2
:102AE700B7A575B7F1740090DE00F075B7A575B797
:102AF700F1740090E000F075B7A575B7F174009018
:102B0700E200F075B7A575B7F1740090E400F075B1
:102B17008F01750A00750900AE09AF0A74FFC39FDC
:102B270074019E402475B7A575B7F190004E120049
:102B37001EE0FC90DE0012001EECF0780A740126FD
:102B4700F6500418E436F650CF750A00750900AE42
:102B570009AF0A74FFC39F74019E402475B7A5751A
:102B6700B7F190024E12001EE0FC90E00012001E2A
:102B7700ECF0780A740126F6500418E436F650CFC4
:102B8700750A00750900AE09AF0A74FFC39F740187
:102B97009E402475B7A575B7F190044E12001EE04C
:102BA700FC90E20012001EECF0780A740126F65041
:102BB7000418E436F650CF750A00750900AE09AF60
:102BC7000A74FFC39F74019E402475B7A575B7F1BA
:102BD70090064E12001EE0FC90E40012001EECF07E
:102BE700780A740126F6500418E436F650CF758F2C
:102BF7000075F51175B62075D940D2AF743A9007B4
:102C07004EF022900788E0B4AA028003022D47C243
:102C1700AF75D90075B62275F522758F0375B7A5FF
:102C270075B7F1740090D600F075B7A575B7F17454
:102C37000090D800F075B7A575B7F1740090DA0069
:102C4700F075B7A575B7F1740090DC00F0758F01CA
:102C5700750A00750900AE09AF0A74FFC39F7401B6
:102C67009E402475B7A575B7F190004E12001EE07F
:102C7700FC90D60012001EECF0780A740126F6507C
:102C87000418E436F650CF750A00750900AE09AF8F
:102C97000A74FFC39F74019E402475B7A575B7F1E9
:102CA70090024E12001EE0FC90D80012001EECF0BD
:102CB700780A740126F6500418E436F650CF750AE0
:102CC70000750900AE09AF0A74FFC39F74019E40E7
:102CD7002475B7A575B7F190044E12001EE0FC905D
:102CE700DA0012001EECF0780A740126F650041878
:102CF700E436F650CF750A00750900AE09AF0A74BD
:102D0700FFC39F74019E402475B7A575B7F1900660
:102D17004E12001EE0FC90DC0012001EECF0780A58
:102D2700740126F6500418E436F650CF758F0075F7
:102D3700F51175B62075D940D2AF743A90074EF0A9
:102D470022C2AF75D90075F522750A00750900AE64
:102D570009AF0A74FFC39F74019E401F90EE0012D3
:102D6700001EE493FC90004E12001EECF0780A74EB
:102D77000126F6500418E436F650D4750A00750992
:102D870000AE09AF0A74FFC39F74019E401F90F005
:102D97000012001EE493FC90024E12001EECF07825
:102DA7000A740126F6500418E436F650D4750A0062
:102DB700750900AE09AF0A74FFC39F74019E401FD7
:102DC70090F20012001EE493FC90044E12001EECD9
:102DD700F0780A740126F6500418E436F650D475D4
:102DE7000A00750900AE09AF0A74FFC39F74019EFC
:102DF700401F90F40012001EE493FC90064E120050
:102E07001EECF0780A740126F6500418E436F650E2
:102E1700D475F51175D940D2AF22C2AF75D90075F7
:102E2700F522750A00750900AE09AF0A74FFC39F42
:102E370074019E401F90E60012001EE493FC900070
:102E47004E12001EECF0780A740126F6500418E4BE
:102E570036F650D4750A00750900AE09AF0A74FF3B
:102E6700C39F74019E401F90E80012001EE493FC6C
:102E770090024E12001EECF0780A740126F65004F8
:102E870018E436F650D4750A00750900AE09AF0A82
:102E970074FFC39F74019E401F90EA0012001EE456
:102EA70093FC90044E12001EECF0780A740126F68B
:102EB700500418E436F650D4750A00750900AE09B7
:102EC700AF0A74FFC39F74019E401F90EC0012006D
:102ED7001EE493FC90064E12001EECF0780A740173
:102EE70026F6500418E436F650D475F51175D94016
:102EF700D2AF22C2AF75D90075F522750A007509E0
:102F070000AE09AF0A74FFC39F74019E401F90DE95
:102F17000012001EE493FC90004E12001EECF078A5
:102F27000A740126F6500418E436F650D4750A00E0
:102F3700750900AE09AF0A74FFC39F74019E401F55
:102F470090E00012001EE493FC90024E12001EEC6B
:102F5700F0780A740126F6500418E436F650D47552
:102F67000A00750900AE09AF0A74FFC39F74019E7A
:102F7700401F90E20012001EE493FC90044E1200E2
:102F87001EECF0780A740126F6500418E436F65061
:102F9700D4750A00750900AE09AF0A74FFC39F74A0
:102FA700019E401F90E40012001EE493FC90064E21
:102FB70012001EECF0780A740126F6500418E43665
:102FC700F650D475F51175D940D2AF22C2AF75D975
:102FD7000075F522750A00750900AE09AF0A74FF7E
:102FE700C39F74019E401F90D60012001EE493FCFD
:102FF70090004E12001EECF0780A740126F6500479
:1030070018E436F650D4750A00750900AE09AF0A00
:1030170074FFC39F74019E401F90D80012001EE4E6
:1030270093FC90024E12001EECF0780A740126F60B
:10303700500418E436F650D4750A00750900AE0935
:10304700AF0A74FFC39F74019E401F90DA001200FD
:103057001EE493FC90044E12001EECF0780A7401F3
:1030670026F6500418E436F650D4750A00750900A0
:10307700AE09AF0A74FFC39F74019E401F90DC0026
:1030870012001EE493FC90064E12001EECF0780A24
:10309700740126F6500418E436F650D475F5117508
:1030A700D940D2AF22E51464046006E59964FF6055
:1030B700028031A20F4004D20F8027E51460087404
:1030C700E62514900023F0E513600874F0251390AB
:1030D7000023F0E514B4010280FE75140075130097
:1030E700C20F8002C20FE514903A07F828287375BB
:1030F7001400E599B4FF03751301E599B4FE037550
:103107001302E599B4FD03751303E599B4FC037540
:103117001304E599B4FA03751305E599B4FB06752D
:103127001401120481E599B4F90675140412048197
:10313700E599D394E54007E599C394F040028016DA
:103147008599157514027E017F00E515C394E61273
:103157003F9E8E0D8F0E900786E4F0A3F0E599D37E
:1031670094C44007E599C394E640028028859915E1
:1031770075140374E5C39515F50E750D00AE0DAF07
:103187000E903A6412002EE493F874019390078628
:10319700C8F0A3C8F0D29902361B900786E0FEA3B9
:1031A700E0FFEFC39400EE94054009EFD394FFEEE0
:1031B70094064013900786E0FEA3E0FF90004E12AE
:1031C700001EE599F0800385996C90078612000E22
:1031D700900786E0FEA3E0FFEFB40106EEB4070216
:1031E700800302342B90074EE0B43C028003023484
:1031F7002BA20AB35005A20BB3400302331EC29C95
:1032070090007AE090078CF0900057E090078DF0DF
:10321700900062E090078EF0900063E090078FF0D7
:10322700900074E0900790F090007CE0900791F098
:1032370090007DE0900792F0900080E0900793F077
:10324700900081E0900794F090013AE0900795F0A4
:1032570090013BE0900796F090013CE0900797F0D3
:10326700900090E0900798F0900091E0900799F017
:10327700900092E090079AF0900093E090079BF0FF
:10328700900094E090079CF0900095E090079DF0E7
:10329700900096E090079EF0900097E090079FF0CF
:1032A700900099E09007A0F090009AE09007A1F0B5
:1032B70090009BE09007A2F090009CE09007A3F09D
:1032C7007400900082F01200C974AB900788F01266
:0A32D70027A574AA900788F0E558B7
:063A07000230F60231A1BD
:1032E100903A28F82828738012122850800D12294C
:0B32F1008E8008122ACC8003122C0AE9
:0F3A28000232E80232EA0232EF0232F40232F9DD
:1032FC00900788E4F090013AE0700C90013BE0708C
:10330C000690013CE060028004C20A8002D20A02EC
:10331C003420C29C900078E0900789F090005EE029
:10332C0090078AF090005FE090078BF090007AE0B5
:10333C0090078CF0900057E090078DF0900062E0C1
:10334C0090078EF0900063E090078FF0900074E08F
:10335C00900790F090007CE0900791F090007DE059
:10336C00900792F0900080E0900793F0900081E03D
:10337C00900794F090013AE0900795F090013BE0B3
:10338C00900796F090013CE0900797F0900090E049
:10339C00900798F0900091E0900799F0900092E0DF
:1033AC0090079AF0900093E090079BF0900094E0C7
:1033BC0090079CF0900095E090079DF0900096E0AF
:1033CC0090079EF0900097E090079FF0900099E096
:1033DC009007A0F090009AE09007A1F090009BE07D
:1033EC009007A2F090009CE09007A3F0740090006E
:1033FC0082F074AB900788F01227A574AA90078806
:10340C00F012285012298E122ACC122C0AD29C753A
:10341C0099FB80FED29C7514007513007599FB0204
:10342C00361B900786E0FEA3E0FFEF4E70068599F1
:10343C0010750F00900786E0FEA3E0FF74016F4E3D
:10344C00701BAC0FAD10AA0DAB0EED2BFBEC3AFACA
:10345C008A068B0790004E12001EE599F0900786A5
:10346C0012000E900786E0FEA3E0FF74026F4E7010
:10347C000C1200C985159975140075130002361BC2
:10348C00900786E0FEA3E0FF90004E12001EE59927
:10349C00F090078612000E900786E0FEA3E0FFACCA
:1034AC000DAD0E8F028E038C068D07903A9C120088
:1034BC002EE493F9740193FEEAD39EEB99400985AF
:1034CC00159975140075130002361B900786E0FEE3
:1034DC00A3E0FF90004E12001EE599F090078612B3
:1034EC00000E900786E0FEA3E0FFEFB40006EEB4FA
:1034FC000102800302361B90001CE0D394C7400BE2
:10350C0090001CE0C394C8F516801A90001CE0D300
:10351C009463400B90001CE0C39464F516800690F5
:10352C00001CE0F516E51675F002A4FFAEF08F6BEB
:10353C00EF90004E123FB6EFFCE0FDEC9000511204
:10354C003FB6EDFCE0FDEC2DB51602800302360D06
:10355C000FEF90004E123FB6E56BFFE0FCEF9000D2
:10356C0052123FB6ECFFE0FCEFC39CB51602800391
:10357C0002360DE56B900050123FB6E56BFFE0FC98
:10358C00EF900053123FB6ECFFE0FCEF2CB5167138
:10359C00E56B900054123FB6E0C3951690079DF072
:1035AC00E56B900055123FB6E0C3951690079EF060
:1035BC00E56B900058123FB6E0C3951690079FF04C
:1035CC00E56B900059123FB6E0C395169007A0F03A
:1035DC00E56B90005A123FB6E0C395169007A1F028
:1035EC00E56B90005B123FB6E0C395169007A2F016
:1035FC0012271B7599F97518647517001226D78058
:0F360C00FE7599FF7518647517001226D780FE9A
:093A0D0002342E02348C0234D77D
:10361B0022E513903A16F828287302375C90078638
:10362B00E0FEA3E0FF90001212001EE0F599900758
:10363B008612000E900786E0FEA3E0FF74116F4E1A
:10364B00700375130002375C85629902375C900733
:10365B0086E0FEA3E0FF90004E12001EE0F599EF0E
:10366B00B40107EEB4070375130090078612000E22
:07367B0002375C900787E0B5
:0F3A160002362502362802365302365902367E12
:10368200903A37F8282873852499023751852A9968
:10369200023751854499023751854799023751853E
:1036A20051990237518560990237518556990237EF
:1036B20051855899023751756E00900069E0700685
:1036C200900068E060028016A2A44006E56E440401
:1036D200F56EA2A54006E56E4402F56E801A9000D2
:1036E2004AE0B40106E56E4410F56E900049E0B47C
:1036F2000106E56E4420F56EA207B34006E56E446E
:1037020001F56EA209B34006E56E4408F56E856EBA
:1037120099803CA210B340077599FAC2108017A293
:103722000CB3400575990F800B900023E0F599903A
:103732000023E4F0C20C80178542998012854B99D0
:0F374200800D85469980087599FC8003751300EA
:103A370002368902368F02369502369B0236A1027C
:103A470036A70236AD0236B30236B902371502374A
:0D3A57003A02373F02374402374902374E2A
:0B37510090078612000E800312004853
:033A25000237590C
:10375C002290006BE0B4010385241190006BE0B45F
:10376C000203852A1190006BE0B403038544119089
:10377C00006BE0B4040385471190006BE0B40503C3
:10378C0085511190006BE0B4060385561190006BC7
:10379C00E0B4070385581190006CE0FE90006DE0DA
:1037AC00C39E500302383390006BE0D39404402C3A
:1037BC0090006CE0D39511500990006DE0C3951109
:1037CC0050028002D20090006CE0D3951150099009
:1037DC00006DE0C395115002C200804990006BE06F
:1037EC00B4041890006DE0C395115002D200900003
:1037FC006CE0D395114002C200802A90006CE0C3AB
:10380C009511500990006DE0D3951150028002D2B1
:10381C000090006CE0D39511500990006DE0C395B9
:10382C00115002C200807E90006BE0D39404402CB7
:10383C0090006CE0C39511400990006DE0D3951198
:10384C0040028002C20090006CE0C39511400990C8
:10385C00006DE0D395114002D200804990006BE0DE
:10386C00B4041890006CE0C395115002C200900093
:10387C006DE0D395114002D200802A90006CE0C319
:10388C009511400990006DE0D395114002D2009043
:10389C00006CE0D39511400990006DE0C395114088
:1038AC00028002C2002290006EE0B4010385241154
:1038BC0090006EE0B40203852A1190006EE0B40310
:1038CC000385441190006EE0B40403854711900009
:1038DC006EE0B4050385511190006EE0B4060385CB
:1038EC00561190006EE0B4070385581190006FE0FC
:1038FC00FE900070E0C39E500302398890006EE089
:10390C00D39404402C90006FE0D395115009900093
:10391C0070E0C3951150028002D20290006FE0D388
:10392C0095115009900070E0C395115002C20280AD
:10393C004990006EE0B40418900070E0C3951150EB
:10394C0002D20290006FE0D395114002C202802A8D
:10395C0090006FE0C395115009900070E0D3951161
:10396C0050028002D20290006FE0D3951150099062
:10397C000070E0C395115002C202807E90006EE090
:10398C00D39404402C90006FE0C395114009900033
:10399C0070E0D3951140028002C20290006FE0C328
:1039AC0095114009900070E0D395114002D202802D
:1039BC004990006EE0B4041890006FE0C39511506C
:1039CC0002C202900070E0D395114002D202802A0C
:1039DC0090006FE0C395114009900070E0D39511F1
:1039EC004002D20290006FE0D39511400990007014
:0B39FC00E0C3951140028002C20222CD
:093FB6002582F5825002058322E8
:10002E00EF2F500205832582F582E5833E2EF58360
:01003E00229F
:08000300C3EF9DFFEE9CFE22FD
:08003F000806B60002180622B3
:0D000E00A3E004F07006123FACE004F02205
:083FC8000816B6FF02181622CC
:0E3F9000048007C3CE13CECF13CFD5E0F622A8
:103DA800BC000FBE0008ED8FF084FFADF022E4FEEA
:103DB800FF22BE000DEF60FE54F0606F20E70302A3
:103DC8003E5EEAC0E0EBC0E078017A0075F001EEF3
:103DD80020E710EF25E0FFEE33FE0AC5F023C5F01B
:103DE80030E7F0EA5407F9096A7A007B00600108B5
:103DF800C3EC9E40167004ED9F4010ED9FFDEC9EB5
:103E0800FCE5F0CA4ACA03F5F08005E5F003F5F0D1
:103E1800C3EE13FEEF13FFD9D77908CACBCAD8D09F
:103E2800EAFEEBFFD0E0FBD0E0FA22EC8FF084FC56
:103E3800ED54F045F0C48FF084FEEDC454F045F025
:103E4800C48FF084FDEEC4FE54F02DFFEE540F3CF9
:103E5800FEADF07C0022790078008FF0EC7E08201F
:103E6800E70DC3CD33CD33C933C9C833C8DEF084B9
:103E780049F9E5F08FF0BE00E6FD7C00E9FFE8FEB9
:013E88002217
:0E3F9E00F88FF0A4FFE5F0CE88F0A42EFE22EE
:103F7000600D782B023F7A007830D8FED5E0F82229
:103F8000EEC0E07E00123DA8EFFDEEFCD0E0FE2288
:03000B00023F1F92
:03001B00023F3A67
:03002B00023F553C
:03000000023FBFFD
:093FBF0075817275D0000207FD46
:0B001E00E5822FF582E5833EF583228A
:0A3FAC000582D582021583158222DA
:103F1F00C0E0C0F0C083C082C0D075D0001207F2DD
:103F2F00D0D0D082D083D0F0D0E032C0E0C0F0C08B
:103F3F0083C082C0D075D0001207F5D0D0D082D008
:103F4F0083D0F0D0E032C0E0C0F0C083C082C0D0D8
:103F5F0075D0001207F8D0D0D082D083D0F0D0E047
:013F6F00321F
:00000001FF
